:020000040800F2
:10000000B008002099190008750900087709000850
:100010007B0900087F090008830900080000000030
:100020000000000000000000000000008709000838
:1000300089090008000000008B0900088D090008EC
:10004000B3190008B3190008B3190008B319000860
:10005000B3190008B3190008B3190008B319000850
:10006000B3190008B3190008B3190008B319000840
:10007000B3190008B3190008B3190008B319000830
:10008000B3190008B3190008B3190008B319000820
:10009000B3190008B3190008B3190008B319000810
:1000A000B3190008B3190008B3190008B319000800
:1000B000B31900082D150008B31900082F15000802
:1000C0001D1700087117000815190008B31900085A
:1000D000B3190008EF120008B3190008B31900089B
:1000E000B3190008B3190008B3190008B3190008C0
:1000F000B3190008B3190008B3190008B3190008B0
:10010000B3190008B3190008B3190008B31900089F
:10011000B3190008B3190008B3190008B31900088F
:10012000B3190008B3190008B3190008B31900087F
:1001300000F002F800F05FF80AA090E8000C82449A
:100140008344AAF10107DA4501D100F054F8AFF277
:10015000090EBAE80F0013F0010F18BFFB1A43F0A5
:100160000103184788430000A84300000A444FF0E9
:10017000000C10F8013B13F0070408BF10F8014B06
:100180001D1108BF10F8015B641E05D010F8016B4B
:10019000641E01F8016BF9D113F0080F1EBF10F8AF
:1001A000014BAD1C0C1B09D16D1E58BF01F801CBD2
:1001B000FAD505E014F8016B01F8016B6D1EF9D555
:1001C0009142D6D37047000000230024002500266A
:1001D000103A28BF78C1FBD8520728BF30C148BFAA
:1001E0000B607047642904F06180002070471FB5E0
:1001F0001FBD10B510BD04F047F91146FFF7F7FF1A
:1002000000F0D3FA04F065F903B4FFF7F2FF03BC82
:1002100001F012F810B50020FA49087035E000F03E
:10022000F7FC582000F0A9FD02E0582000F0A5FDE1
:1002300000F030FD0028F8D1F349F24A1278885CCA
:1002400000F09BFD05E0F049EE4A1278885C00F072
:1002500094FD00F01FFD0028F5D1EC49E94A127821
:10026000885C00F08AFD05E0E849E64A1278885C7F
:1002700000F083FD00F00EFD0028F5D100F0E8FC51
:10028000E0480078401CDF490870DE4800781828F4
:10029000C5DB10BDFF20DE49487688760020D949AD
:1002A000087016E0FF20DA49D64A12788854FF21F8
:1002B000D748401DD74A127881540A30D54A12785F
:1002C0008154D44A12788154CE480078401CCD49DC
:1002D0000870CC4800780528E4DB704710B5012190
:1002E000022002F038FE10BD08B50220ADF8000073
:1002F00003208DF8020010208DF803006946C648DF
:1003000002F03EF908BD0EB50121C44803F084FD9A
:100310004FF4FA70ADF8040048F69F40ADF80000C5
:100320000020ADF80600ADF802006946BB4802F0B7
:100330003DFF01221146B94803F0AFFA0121B74849
:1003400003F090FA0EBD10B502F08AFC012002F015
:100350000CFD00BF212002F0C6FC0028FAD00020CE
:1003600002F023FD002002F032FD4FF4806002F025
:1003700025FD022001F0C6FD102001F0D7FD4FF44D
:100380002011002002F0F4FC012002F0FDFC00BF6F
:10039000392002F0A8FC0028FAD0022002F0F7FC75
:1003A00000BF02F0FDFC0828FBD101211C2002F057
:1003B000C5FD0121084602F0C1FD10BD70B505461E
:1003C0000C4645F2555002F02BFC284602F02BFC5F
:1003D000204602F02BFC02F02CFC02F02FFC70BD3A
:1003E00010B502F026FC10BD10B58D480078C0B1E4
:1003F000012817D0022802D0032816D109E000F006
:1004000088FE01208649087040F6B83085490860AA
:100410000BE000F0ADFB00208349086080490870C4
:1004200003E002E000F0FCFD00BF00BF10BD10B50E
:1004300000F0EEFBBA2000F0A0FC00F02BFC002046
:1004400000F09BFC00F026FC0446214677A003F058
:10045000EDFE14B940F28F3010BD4FF4A350FBE70E
:1004600070B500F0D5FB702000F087FC02E0702032
:1004700000F083FC00F00EFC0028F8D100F07DFCB9
:1004800002E0002000F079FC00F004FC0028F8D124
:1004900000F0DEFB00F0BCFB712000F06EFC02E01F
:1004A000712000F06AFC00F0F5FB0028F8D15549F6
:1004B00008700BE0012000F08BFC5F49514A127874
:1004C000885450480078401C4E4908704D480078C8
:1004D0002028EFDB002000F07BFC574981F820004A
:1004E00000F0B6FB5448807818B153488078FF2854
:1004F00004D1514880784649487681E04E4880785A
:1005000005287DDC4C488078414948760846407E85
:10051000052801DD0520487600203E49087069E085
:100520003C4C247804EB44046400241D424D2D5DB2
:10053000384C247804EB44046400E41C3E4E345DE3
:1005400004F00F0445EA0420324C247804EB440400
:100550006400A41D35462D5D2E4C247804EB440424
:100560006400641D345D04F00F0445EA0421294C45
:10057000247804EB44046400E41C35462C5DA2118D
:10058000244C247804EB44046400641D2C5D231186
:10059000B0F5487F01DD4FF44870B1F5F07F01DD23
:1005A0004FF4F07100B9012001B90121C0F5487480
:1005B000A0B2C1F5F074A1B2154D164E3678A8550B
:1005C000050A134C641D134E3678A555641D114E53
:1005D0003678A1550D0A641D0E4E3678A5550F3C90
:1005E000A27614340B4D2D7863550A480078401CD0
:1005F000084908700648407E0649097888428FDC21
:1006000070BD000000000020080000202000002035
:100610006B01002001000020001001400004004098
:100620001A010020080100208C01214261636B3D0A
:100630002025640D0A0000004001002070B5002054
:10064000B9490870B94908700122B94948F24E10F9
:1006500000F024FCB648007818B1B5480078FF28AF
:100660001DD1B4480078401CB24908700846007893
:10067000012808D100F0A0FD0122AD4948F24E103A
:1006800000F00CFC0FE0AB480078042806DD0420E5
:10069000A8490870A6480078A74948767EE000205F
:1006A000A449087000BFA248007800F0800000282C
:1006B00074D09F48007800F00F0000286EDD9C4841
:1006C000007800F00F009C4948760846407E0528D7
:1006D00001DD052048769848407EC000401CC2B22B
:1006E000934948F24E1000F0D9FB00208F49087062
:1006F0004EE08E4B1B78DB005B1C8D4CE25C8B4B21
:100700001B78DB009B1CE45C884B1B78DB00DB1C4C
:10071000874DEB5C44EA0320844B1B78DB001B1DF8
:100720002C46E45C814B1B78DB005B1DEB5C44EAF0
:100730000321B0F5487F01DD4FF44870B1F5F07F3B
:1007400001DD4FF4F07100B9012001B90121C0F5BC
:10075000487398B2C1F5F07399B2774B734D2D7809
:100760005855040A5B1D714D2D785C555B1D6F4D0E
:100770002D7859550C0A5B1D6C4D2D785C555B1D11
:100780006A4C24781A5569480078401C67490870FB
:100790006948407E654909788842AADC0122674998
:1007A00048F24E1000F04CFB70BDB0B0B82102A86A
:1007B00003F0B8FDFFF7C7FDFFF790FD4FF4E13000
:1007C00000F049FD5EA003F031FD7D2002F08BFAC0
:1007D00030B102F0F1FB04215FA003F027FD02E03D
:1007E00002206049087000F0CFFB4FF47A710620B8
:1007F000FFF7E4FD00F0A8FC00F00AFD00F0BCFDEE
:1008000000F005FE00F0C0FB322000F0D5FC012115
:10081000082002F093FB0320ADF8040010208DF8AF
:10082000070003208DF8060001A94F4801F0A8FE3B
:1008300001214D4801F051FF02214B4801F04DFFCD
:1008400000F0CDF90220ADF8040028208DF8070053
:1008500001A9454801F094FE0221434801F03FFF01
:10086000FFF718FDFFF7D6FC01213F4801F037FFE5
:100870000A2000F0A1FC01213B4801F02EFF3220AC
:1008800000F09AFCFFF7D3FD40F28F31884226D169
:1008900002208DF80800012202A948F2400000F071
:1008A000CFFA022202A948F2470000F0F7FA9DF8B9
:1008B0000800502802D0012000F039FB0A2000F087
:1008C0007BFC00208DF80800012202A948F24000BC
:1008D00000F0B6FA40F28F302449086003E04FF48C
:1008E000A350224908601DE021480078012817D153
:1008F00000201F490870012000F05EFCFFF774FD26
:100900001A48006840F28F31884202D1FFF796FE04
:1009100006E016480068B0F5A35F01D1FFF7A0FD1F
:10092000FFF75EFDE0E7000000000020010000206E
:1009300040010020380000206B0100203900002019
:10094000444652303637382056322E305F323032FD
:1009500031303431320D0A0057445420525354255B
:10096000640D0A001A010020000C01400400002060
:100970001E010020704700BFFEE700BFFEE700BF7A
:10098000FEE700BFFEE77047704770477047000002
:100990000CB50020019000906C48006840F4803055
:1009A0006A49086000BF6948006800F400300090A0
:1009B0000198401C0190009818B90198B0F5A06FFB
:1009C000F1D16248006800F4003010B101200090BD
:1009D00001E0002000900098012843D15C480068A5
:1009E00040F010005A4908600846006820F00300F3
:1009F00008600846006840F00200086053484068FC
:100A0000524948600846406848600846406840F4DB
:100A1000806048600846406820F47C1048600846C2
:100A2000406840F4E81048600846006840F0807074
:100A3000086000BF4548006800F000700028F9D049
:100A40004248406820F0030040494860084640683A
:100A500040F00200486000BF3C48406800F00C00D5
:100A60000828F9D10CBD10B5FFF792FF10BD10B5E5
:100A70003648006840F00100344908600846406884
:100A80003449084031494860084600683249084006
:100A90002E4908600846006820F480200860084657
:100AA000406820F4FE0048604FF41F008860FFF7A4
:100AB000DAFF4FF000602949086010BD10B5002131
:100AC00000200022214B5B6803F00C0121B10429B6
:100AD00006D0082928D107E0214B224C236027E0CB
:100AE0001F4B204C236023E0184B5B6803F470100D
:100AF000164B5B6803F48032022303EB904022B96B
:100B0000194B4343174C23600DE0104B5B6803F413
:100B1000003323B1144B4343124C236003E0104BCA
:100B20004343104C236003E00D4B0E4C236000BF89
:100B300000BF064B5B68C3F303130C4CE15C094B2D
:100B40001B68CB40074C236010BD00000010024022
:100B5000002002400000FFF8FFFFF6FE08ED00E075
:100B600000127A003C00002000093D0040000020F7
:100B700008B50121042002F0E1F90820ADF80000D9
:100B800010208DF8030003208DF8020069460F48FD
:100B900001F0F6FC0121082002F0D0F90120ADF8A7
:100BA000000010208DF8030003208DF80200694634
:100BB000074801F0E5FC0220ADF8000048208DF860
:100BC00003006946024801F0DBFC08BD0008014053
:100BD000000C014010B5042000F0CAFA10BD08B5A1
:100BE0000121042002F0AAF94FF44060ADF80000A2
:100BF00010208DF8030003208DF8020069468D480F
:100C000001F0BEFC4FF440618A4801F066FD08BD6A
:100C100010B58848001D006820F470608549091DE2
:100C200008600846006840F440700860012082496E
:100C300008608249C1F8AC01FFF7CCFF00207E4973
:100C40000860FFF7C7FF00207C49C1F8AC0110BD68
:100C500010B57848001D006820F470607549091DC2
:100C600008600846006840F440700860002072493F
:100C7000091D08607149C1F8A801FFF7ABFF012009
:100C80006D49091D0860FFF7A5FF01206B49C1F8F8
:100C9000A80110BD10B500246648001D006820F4AE
:100CA00070606449091D08600846006840F40060EF
:100CB000086001206049086000F05AFA01205F498D
:100CC000C1F8AC0100F054FA07E0601CC4B2642C17
:100CD00003DDFFF7BDFF012010BD574880380068D5
:100CE0000028F2D15449091D086000BFF4E710B58F
:100CF00000205149091D08604E48001D006820F47D
:100D000070604C49091D08600846006840F4407056
:100D1000086000204949C1F8A801FFF75BFF0120E6
:100D20004549091D0860FFF755FF00204349C1F8F8
:100D3000AC0110BD10B500203F49091D08603D48B9
:100D4000001D006820F470603A49091D08600846DB
:100D5000006840F44070086001203849C1F8A801DB
:100D6000FFF738FF01203449091D0860FFF732FF03
:100D700000203249C1F8AC0110BD70B504462D48C1
:100D8000001D006820F470602A49091D08600846AB
:100D9000006840F44070086000202749091D086081
:100DA000002512E0E009244908606006040E0120D5
:100DB0002249C1F8AC01FFF70DFF00201E49091DB3
:100DC0000860FFF707FF681CC5B2082DEADB70BD9D
:100DD00070B5054600241748001D006820F47060B7
:100DE0001449091D08600846006840F40060086066
:100DF000002614E000201049091D08600A2000F0B8
:100E0000B7F901200D49C1F8AC016006040E0A488B
:100E10008038006808B1601CC4B2701CC6B2082ECD
:100E2000E8DB15B9FFF786FF01E0FFF760FF20461A
:100E300070BD000000080140A801214200002142CD
:100E40002DE9F04104460E4617464FF00008FFF723
:100E5000DFFEBA20FFF791FFFFF71CFF2012FFF71C
:100E60008CFFFFF717FFE0B2FFF787FFFFF712FFD6
:100E700000250BE0705DFFF780FFFFF70BFF80465A
:100E8000B8F1000F00D003E0681CC5B2BD42F1DB31
:100E900000BFFFF7DDFE4046BDE8F0812DE9F041DF
:100EA00004460F461646FFF7B3FEBA20FFF765FF6C
:100EB00002E0BA20FFF761FFFFF7ECFE0028F8D14F
:100EC0002012FFF75AFF02E02012FFF756FFFFF74C
:100ED000E1FE0028F8D1E0B2FFF74FFF02E0E0B2F8
:100EE000FFF74BFFFFF7D6FE0028F8D1FFF790FE83
:100EF000BB20FFF742FF02E0BB20FFF73EFFFFF7FA
:100F0000C9FE0028F8D100250BE0711EA94201D0CE
:100F1000012100E000210846FFF75AFF7855681CC0
:100F2000C5B2B542F1DBFFF793FEBDE8F08138B5FD
:100F30000546002400208DF800008DF8015000BF08
:100F400009E09DF800000F49095D0844C0B28DF822
:100F50000000601CC4B2B82CF3D39DF80000C0435D
:100F6000401CC0B28DF80000B822064948F2470084
:100F7000FFF766FF0222694648F2FF00FFF760FFB5
:100F8000002038BD5000002000B587B0012140F29C
:100F9000052001F0D3FF4FF4004001F033FF0120A2
:100FA000ADF8180000208DF81B0003208DF81A0002
:100FB00006A9614801F0E4FA002001908DF80800CC
:100FC0008DF809004FF46020039000200490012068
:100FD0008DF8140001A9594800F093FD0723012260
:100FE0000021564800F025FE0121544800F0B5FDCF
:100FF000524800F0D4FD00BF504800F0D5FD002855
:10100000FAD14E4800F0DAFD00BF4C4800F0DBFD9D
:101010000028FAD10121494800F0DFFD07B000BDEA
:1010200070B50024002510E00121444800F0D5FDF2
:1010300000BF0221414800F041FF0028F9D03F489D
:1010400000F05EFE0444681CC5B2082DECDBE40829
:101050003B480068001B19280CD9A4F214504FF427
:10106000616148434FF40C71B0FBF1F035490880E1
:1010700033480460204670BD30B589B005460C4643
:101080000121084601F067FF0121052001F056FF0C
:101090000820ADF8200018208DF8230003208DF8DB
:1010A000220008A9244801F06BFAADF81850ADF8F9
:1010B00014400020ADF81A00ADF8160005A94FF055
:1010C000804002F073F87020ADF804000120ADF804
:1010D00006000420ADF808000220ADF80C00002046
:1010E000ADF80E004FF48070ADF810000020ADF8A0
:1010F000120001A94FF0804002F06FF90821C806E4
:1011000002F0FFFC00214FF0804002F0ABFB09B081
:1011100030BD10B5092140F60F60FFF7ADFF4FF469
:10112000E160084908800121C00602F09BFB012113
:10113000880702F0A3FB10BD000801400024014015
:1011400008010020400000402D4800682D49B0FBF8
:10115000F1F02D4908700846007800EB4001C1EB22
:10116000C0104FF6FF7101EAC0002849088070479F
:101170000146254A12784A434FF0E0235A61002283
:101180009A611A46126942F001021A6100BF4FF0DB
:10119000E022106900F001021AB100F48032002A46
:1011A000F5D04FF0E022126922F001024FF0E02367
:1011B0001A6100229A6170470146144A12884A4314
:1011C0004FF0E0235A6100229A611A46126942F0F8
:1011D00001021A6100BF4FF0E022106900F0010225
:1011E0001AB100F48032002AF5D04FF0E0221269E3
:1011F00022F001024FF0E0231A6100229A61704749
:101200003C00002000127A000C0100200E0100209A
:1012100008B54FF4A06000F0DFFB1D208DF8000042
:1012200000208DF8010001208DF802008DF80300E8
:10123000684600F0D6FB08BD014600BF704700BFFE
:10124000494A128802F04002002AF9D0C2B2464B45
:101250001B1D1A80704710B586B00446012144F268
:10126000040001F06BFE4FF40070ADF81400032091
:101270008DF8160018208DF8170005A93B4801F0DD
:101280007FF94FF48060ADF8140004208DF817004A
:1012900005A9364801F074F925208DF800000320D7
:1012A0008DF801008DF8020001208DF803006846DA
:1012B00000F097FB01940020ADF80800ADF80A009B
:1012C000ADF80C00ADF810000C20ADF80E0001A92F
:1012D000254802F0E8FD012240F22551224802F0A3
:1012E0007AFE0121204802F06AFE06B010BD10B55A
:1012F00040F225511C4802F053FF10B31A4802F087
:10130000CFFEC4B21A48008800F40040C8B918489B
:10131000008800F4804060B10A2C03D000201449FA
:10132000088020E01248008840F4004010490880FE
:1013300019E00D2C06D10E48008840F480400C497D
:10134000088010E00A480088C0F30D0009490C54D9
:1013500007480088401C0649088008460088C728BE
:1013600001DD0020088010BD003801400008014068
:10137000140100208601002000B587B001218805F6
:1013800001F0E9FD0121082001F0D8FD4FF4406093
:10139000ADF8180003208DF81A001C208DF81B00F2
:1013A00006A9FE4801F0ECF8FD4802900020ADF8D7
:1013B0000C004BF6FF70ADF80E00FA480088ADF84F
:1013C00010004FF48060ADF812000001ADF8140079
:1013D00002A9F54801F03BFA01224FF4E061F2481E
:1013E00001F01EFB21208DF8040001208DF805007E
:1013F00000208DF8060001208DF8070001A800F0FC
:10140000F0FA0121E84801F0A0FA07B000BD00B5EC
:1014100087B00121480501F09EFD0121082001F05F
:101420008DFDC020ADF8180003208DF81A001C2097
:101430008DF81B0006A9D94801F0A2F8D8480290FF
:101440000020ADF80C004BF6FF70ADF80E00D74849
:101450000088ADF810004FF48060ADF81200000174
:10146000ADF8140002A9D24801F0F1F901224FF4BD
:10147000E061CF4801F0D4FA1F208DF8040001206C
:101480008DF8050000208DF8060001208DF807007A
:1014900001A800F0A6FA0121C54801F056FA07B0EC
:1014A00000BD10B50446C349204601F075FB208BF2
:1014B00010BD10B50446BF490E31204601F06CFB4B
:1014C0000121204601F041FA10BD10B5B848FFF7E0
:1014D000E8FFFFF79CFF10BD10B50446B248FFF7C8
:1014E000E0FFB5480178B04801F0A3FA10BD10B58F
:1014F000AF48FFF7D6FFB148007840B90120AF49A7
:101500000870AF48417EAA4801F093FA0DE0002030
:10151000AC490870AC480078401EA94A521D105CC6
:1015200040F08001A24801F084FA10BD704710B568
:10153000A6499F4801F053FB18B1A4499C4801F00B
:1015400069FB9B4801F01BFBA14A811A904271D0B4
:101550001ADCA04AA0EB020190426CD00DDC1028EE
:101560007FD0B0F5806F68D0B0F1021F28D0A0F511
:1015700000304038002870D126E001296ED00729BC
:101580006DD03F29F7D1C1E0934A881A914267D0C4
:1015900009DC022971D0A1F57F41FE3900296BD009
:1015A0000229E8D1B3E08D490844002876D0B0F58F
:1015B000E00F74D0A0F5E80080380028DBD1A1E06E
:1015C0007B48FFF76EFFA7E0794801F034FA8449C1
:1015D00008700020834908700120784908700020B5
:1015E000814908707E480078022803D100207349A1
:1015F000087031E07A480078032803D1012072494D
:10160000087029E076480078092803D102206E4945
:10161000087021E0724800780F2803D103206A493E
:10162000087019E06E480078152807D10420664933
:10163000087011E019E067E013E05DE068480078A9
:101640001B2803D105206049087005E06448007834
:10165000FF2801D1FFF739FF5EE05CE055E059E07B
:1016600057E05348FFF725FF56E0FFF740FF012002
:101670005E49087050E000E04AE05248007878B9CE
:1016800051480078401E4E4A115C494801F0D1F99A
:101690004C480078401C4B4908702CE033E030E0A7
:1016A00048480078012816D147480078401E444A2F
:1016B0001432135C44480078401E521F105C63F3E0
:1016C0001F10C1B23A4801F0B4F93E480078401CFE
:1016D0003C4908700FE03B48007802280BD13A489B
:1016E0000078401E364A0A32115C314801F0A1F9F7
:1016F0000020344908700FE034492D4801F08AFA7F
:101700000AE009E008E007E006E005E004E003E0A5
:1017100002E001E000E000BF00BF10BD10B5344999
:10172000234801F05CFA10BB3249214801F057FA16
:10173000E8B931491E4801F052FAC0B92F491C4896
:1017400001F04DFA98B92149194801F048FA20B141
:101750001E49174801F05EFA09E02949144801F0D2
:101760003EFA20B94FF00121114801F038FA10BDBE
:1017700010B516490C4801F032FA18B113490A485D
:1017800001F048FA084801F0FAF9114A811A90422A
:1017900070D04FDC0F4AA0EB020133E0000C014097
:1017A000A08601001801002000580040160100200A
:1017B0000054004002000010200100202101002000
:1017C0006B010020250100201B0100200004000106
:1017D0008200060001000300020001008400F5FF02
:1017E0001F01002024010020270100201E010020ED
:1017F000008000010040000100100001000800010D
:1018000000020001904279D00DDC102862D0B0F5C2
:10181000806F6BD0B0F1021F28D0A0F500304038A7
:10182000002874D127E0012969D007296ED03F290B
:101830006DD165E04C4A881A914266D009DC0229D4
:1018400053D0A1F57F41FE3900295DD002295ED138
:1018500059E04649084400284FD0B0F5E00F4AD07F
:10186000A0F5E8008038002851D145E04048FFF756
:1018700018FE4DE032E03E4801F0DDF83D490870C9
:1018800008460078012802D13B49087021E0394818
:101890000078802803D1C3203749087019E0354803
:1018A0000078822803D185203349087011E031483F
:1018B000007804280DD02F480078FF2803D102209B
:1018C0002E49087005E02B48007810B903202B49F9
:1018D00008701DE02648FFF7ECFD19E02648007867
:1018E000FFF7FAFD14E009E000E011E02449204888
:1018F00001F090F90CE00BE00AE009E008E007E0F5
:1019000006E004E002E003E002E001E000E000BFE6
:1019100000BF10BD10B51B49154801F060F910BBA0
:101920001949134801F05BF9E8B91849104801F06A
:1019300056F9C0B916490E4801F051F998B9104945
:101940000B4801F04CF920B10D49094801F062F94A
:1019500009E01049064801F042F920B94FF0012191
:10196000034801F03CF910BD020001008400F5FFBE
:10197000005800401F010020200100201A01002013
:10198000000400010080000100400001001000017F
:10199000000800010002000109488047094800478B
:1019A000FEE7FEE7FEE7FEE7FEE7FEE7FEE7FEE70F
:1019B000FEE7FEE704480549054A064B704700006C
:1019C0006F0A000831010008B0020020B0080020B2
:1019D000B0040020B004002031490143314A1160B5
:1019E000704770B5002100230F22C47804B32D4C3A
:1019F000246804F4E064C4F5E064210AC1F104033E
:101A0000CA40447804FA03F1847814402143090160
:101A1000254C0678A155047804F01F050124AC403C
:101A200005786D11AD0005F1E025C5F8004109E02C
:101A3000047804F01F050124AC401C4D0678761193
:101A400045F8264070BD1A4A0A400243154B1B1F39
:101A50001A60704739B1134A121D12680243114BC4
:101A60001B1D1A6006E00F4A121D126882430D4BBF
:101A70001B1D1A607047042808D14FF0E021096946
:101A800041F004014FF0E022116107E04FF0E02146
:101A9000096921F004014FF0E02211617047000054
:101AA0000000FA050CED00E000E400E080E100E059
:101AB00080FFFF1F10B50446FA48844208D1012177
:101AC000401501F055FA0021601501F051FA17E0B8
:101AD000F548844208D10121001501F049FA00219E
:101AE000201501F045FA0BE0F048844208D10121AD
:101AF000C80301F03DFA00214FF4004001F038FA2C
:101B000010BD30B50246002000235068E84C20404C
:101B10000D790C6844EA0524204350609068E54C38
:101B20002040D1E902542C434D7944EA4504204336
:101B30009060D06A20F470000C7C641EE4B22343F1
:101B400040EA0350D06230BD002101600171417153
:101B50008160C16001210174704721B1826842F047
:101B60000102826003E0826822F001028260704715
:101B700021B1826842F48072826003E0826822F4BC
:101B800080728260704710B50023CBB21AB14468EE
:101B90001C43446002E044689C43446010BD81687B
:101BA00041F0080181607047014600208A6802F018
:101BB00008020AB1012000E000207047816841F06E
:101BC000040181607047014600208A6802F0040227
:101BD0000AB1012000E00020704721B1826842F480
:101BE000A002826003E0826822F4A0028260704753
:101BF000014600208A6802F480020AB1012000E058
:101C00000020704710B50A4600210023416821F4E6
:101C10006041531E41EA4331416010BD21B1426829
:101C200042F40062426003E0426822F400624260D3
:101C30007047F0B504460D4600200021092D11DD46
:101C4000E068A5F10A0606EB4607072606FA07F143
:101C50008843A5F10A0606EB460603FA06F1084397
:101C6000E0600CE0206905EB4507072606FA07F15E
:101C7000884305EB450603FA06F108432061072A6D
:101C80000FDA606B561E06EB86071F2606FA07F171
:101C90008843561E06EB860605FA06F10843606384
:101CA00022E00D2A0FDA206BD61F06EB86071F26CF
:101CB00006FA07F18843D61F06EB860605FA06F1F9
:101CC0000843206310E0E06AA2F10D0606EB8607E8
:101CD0001F2606FA07F18843A2F10D0606EB8606D9
:101CE00005FA06F10843E062F0BD21B1826842F4D2
:101CF0008012826003E0826822F480128260704762
:101D00000146C86C80B2704766484C300068704726
:101D100021B1426842F48062426003E0426822F4EA
:101D200080624260704721B1426842F48052426052
:101D300003E0426822F48052426070470A46002164
:101D4000816821F4E04111438160704721B18268CC
:101D500042F40042826003E0826822F40042826022
:101D6000704721B1826842F40212826003E0826807
:101D700022F4021282607047014600208A6802F451
:101D800000120AB1012000E000207047F0B50446BF
:101D90001546002000220026092911DDE068A1F186
:101DA0000A0707EB470C072707FA0CF29043A1F14B
:101DB0000A0707EB470703FA07F21043E0600CE05D
:101DC000206901EB410C072707FA0CF2904301EB65
:101DD000410703FA07F210432061A06BC0F30156DC
:101DE000EF1C06F1010CA7EB0C0707EB870C1F2774
:101DF00007FA0CF29043EF1C06F1010CA7EB0C075D
:101E000007EB870701FA07F21043A063F0BD10B596
:101E10000A4600210023816B21F44011531E41EA40
:101E20000351816310BD08B5002300930090009B0F
:101E30000B440093009B1A6008BD08B502460020C1
:101E40000090009201F12800009B18440090009837
:101E5000006880B208BD0A4600214168164B19404F
:101E60001143416070474162826270470A46002117
:101E7000416821F01F0111434160704740B1094999
:101E80000831096841F40001064A0832116007E090
:101E900004490831096821F40001024A083211603E
:101EA000704700000024014000280140003C014030
:101EB000FFFEF0FFFDF7F1FFFFFD3FFF02460020B0
:101EC00013680B400BB1012000E000207047CA43AB
:101ED0000260704770B502460020002300240B12F8
:101EE0005568CEB205EA060415681D4015B10CB15F
:101EF000012000E0002070BD00220A12D3430360DD
:101F00007047000001460020FE4A106800F03800CB
:101F1000084310607047FB49096821F00801F94A3D
:101F2000116011460968014311607047F54909685D
:101F300021F01001F34A1160114609680143116054
:101F40007047F148EF494860F04848607047EE48F4
:101F5000EC494860ED4848607047EA48006940F045
:101F60008000E84908617047E648006940F0800059
:101F7000E449086170470420E249C96801F00101A1
:101F800009B101200EE0DF49C96801F0040109B17F
:101F9000022007E0DB49C96801F0100109B1032004
:101FA00000E00420704700B502460423FFF7E3FF7A
:101FB000034603E0FFF7DFFF0346521E012B01D16A
:101FC000002AF7D102B90523184600BD30B50446F2
:101FD00004254FF43020FFF7E6FF0546042D17D106
:101FE000C848006940F00200C649086108464461DB
:101FF000006940F0400008614FF43020FFF7D3FF44
:102000000546C048006941F6FD710840BD490861B8
:10201000284630BD10B504244FF43020FFF7C3FF2D
:102020000446042C16D1B748006940F00400B549B5
:1020300008610846006940F0400008614FF4302014
:10204000FFF7B1FF0446AF48006941F6FB71084055
:10205000AC490861204610BD00B502460423FFF7D5
:102060008AFF034603E0FFF786FF0346521E012B5B
:1020700001D1002AF7D102B90523184600BD10B5D9
:1020800004244FF43020FFF7E7FF0446042C16D158
:102090009C48006940F004009A49086108460069BC
:1020A00040F0400008614FF43020FFF7D5FF0446B0
:1020B0009448006941F6FB71084092490861204646
:1020C00010BD00208F49C96901F0020109B101204A
:1020D00000E00020704730B5A5250424FFF7F1FF8C
:1020E00000B100254FF43020FFF75DFF0446042CBB
:1020F0003AD18548834988608448886008460069E9
:1021000040F0200008610846006940F04000086186
:102110004FF43020FFF747FF0446042C1BD17948C9
:10212000006941F6DF710840764908610846006998
:1021300040F01000086176480580E002FFF733FFA9
:102140000446052C10D06F48006941F6EF71084035
:102150006C49086108E0052C06D06A48006941F620
:10216000EF71084067490861204630BD78B50646E2
:102170000C46042500200090E802FFF714FF0546F6
:10218000042D24D15F48006940F001005D490861D9
:102190003480E802FFF707FF0546042D10D1B01C7C
:1021A0000090200C00990880E802FFF7FCFE05462D
:1021B0005448006941F6FE7108405249086106E042
:1021C0005048006941F6FE7108404E4908612846B2
:1021D00078BD70B504460D460426F002FFF7E3FE15
:1021E0000646042E11D14748006940F001004549D8
:1021F00008612580F002FFF7D6FE064641480069D7
:1022000041F6FE7108403F490861304670BD70B527
:1022100005460E460424E002FFF7C5FE0446042CE2
:1022200017D13948374988603848886008460069BE
:1022300040F0100008612E80E002FFF7B4FE044673
:10224000052C06D02F48006941F6EF7108402D4952
:102250000861204670BD2DE9F04304464FF6FF7635
:102260003746B046B1460425E443E6B2C4F3072737
:10227000C4F307484FEA1469E802FFF794FE0546E5
:10228000042D49D120481F498860204888600846AD
:10229000006940F010000861FF2E06D01C4808308D
:1022A0000680E802FFF77FFE0546042D08D1FF2FC8
:1022B00006D017480A300780E802FFF774FE05468B
:1022C000042D0AD1B8F1FF0F07D011480C30A0F847
:1022D0000080E802FFF767FE0546042D0AD1B9F138
:1022E000FF0F07D00A480E30A0F80090E802FFF771
:1022F0005AFE0546052D0FD00248006941F6EF71E0
:10230000084007E00020024023016745AB89EFCD7C
:1023100000F8FF1F664908612846BDE8F08330B524
:10232000054604244FF43020FFF73DFE0446042CFC
:1023300041D160485E4988605F488860084600690E
:1023400040F0200008610846006940F04000086144
:102350004FF43020FFF727FE0446042C22D15448C6
:10236000006941F6DF71084051490861084600697B
:1023700040F0100008611DB100205049088002E0C3
:10238000A5204E4908804FF43020FFF70CFE04468C
:10239000052C10D04648006941F6EF7108404449C9
:1023A000086108E0052C06D04148006941F6DF715C
:1023B00008403F490861204630BDF0B505460E464D
:1023C000174604243B483A4988603B488860E0024D
:1023D000FFF7E9FD0446042C19D13548006940F0A7
:1023E00010003349086147F0F8003043284333496F
:1023F000891C0880E002FFF7D6FD0446052C06D0B4
:102400002B48006941F6EF710840294908612046D0
:10241000F0BD2748C069800870472548006A7047AA
:1024200000202349096801F0200109B1012000E0E2
:102430000020704729B11E4A126902431C4B1A61E1
:1024400004E01B4A12698243194B1A617047014626
:102450000020012908D1164AD26902F001020AB10E
:10246000012008E0002006E0114AD2680A400AB1C3
:10247000012000E0002070470D49C860704704202B
:102480000B49C96801F0010109B101200EE00849BA
:10249000C96801F0040109B1022007E00449C968D4
:1024A00001F0100109B1032000E004207047000092
:1024B0000020024023016745AB89EFCD00F8FF1FE4
:1024C00010B50446CC48844208D10121042000F014
:1024D0004FFD0021042000F04BFD46E0C748844238
:1024E00008D10121082000F043FD0021082000F060
:1024F0003FFD3AE0C248844208D10121102000F09B
:1025000037FD0021102000F033FD2EE0BD4884424D
:1025100008D10121202000F02BFD0021202000F017
:1025200027FD22E0B848844208D10121402000F074
:102530001FFD0021402000F01BFD16E0B34884423F
:1025400008D10121802000F013FD0021802000F03F
:102550000FFD0AE0AE48844207D10121801500F04A
:1025600007FD0021A01500F003FD10BD10B50121ED
:10257000084600F0FDFC0021012000F0F9FC10BD30
:102580002DE9F0410246002500260020002300240A
:10259000002791F803C00CF00F0591F803C00CF070
:1025A000100CBCF1000F03D091F802C04CEA0505F5
:1025B00091F800C0BCF1000F31D0146800202BE06E
:1025C0004FF0010C0CFA00F3B1F800C00CEA03065E
:1025D0009E4220D183004FF00F0C0CFA03F7BC434E
:1025E00005FA03FC4CEA040491F803C0BCF1280F7F
:1025F00006D14FF0010C0CFA00FCC2F814C00AE03E
:1026000091F803C0BCF1480F05D14FF0010C0CFA52
:1026100000FCC2F810C0401C0828D1D31460B1F8E7
:1026200000C0BCF1FF0F34DD546800202EE000F143
:10263000080C4FF0010808FA0CF3B1F800C00CEADE
:1026400003069E4221D183004FF00F0C0CFA03F7D2
:10265000BC4305FA03FC4CEA040491F803C0BCF146
:10266000280F05D100F1080C08FA0CF8C2F8148004
:1026700091F803C0BCF1480F07D100F1080C4FF0EE
:10268000010808FA0CF8C2F81080401C0828CED3C4
:102690005460BDE8F0814FF6FF7101800221817026
:1026A0000421C17070470246002093680B400BB1B3
:1026B000012000E0002070470146886880B2704722
:1026C00002460020D3680B400BB1012000E000203F
:1026D00070470146C86880B2704701617047416128
:1026E00070470AB1016100E041617047C160704705
:1026F0004FF480320A43826181618261826982691A
:10270000704702460020434B18684FF6807318400C
:1027100040EA021008433F4B186070473E49C861C9
:102720007047F0B50A46002300240021002500F080
:102730000046B6F1004F02D1364EF16901E0354E48
:102740007168C0F3034583B200F44016B6F5401F2C
:1027500008D121F070612F4E766826F070662D4FFB
:102760007E6012E000F48016B6F5801F06D10326C5
:1027700006FA05F4A14341F0706106E0460D36010A
:1027800003FA06F6B14341F0706122B1460D3601FD
:1027900003FA06F6314300F00046B6F1004F02D1CD
:1027A0001C4EF16101E01B4E7160F0BD30B500229E
:1027B0008B071C0F0F2303FA04F2164B08338C10FF
:1027C00053F824309343134C08348D1044F82530CB
:1027D00023468C1053F824308C07240F00FA04F49D
:1027E00023430C4C08348D1044F8253030BD0A4981
:1027F000DC3108607047000000080140000C014017
:10280000001001400014014000180140001C01406C
:1028100000200140000001400000204210B50446A5
:10282000F748844209D10121480500F0AEFB0021A0
:102830004FF4001000F0A9FB08E00121880500F02A
:10284000A4FB00214FF4800000F09FFB10BD2DE998
:10285000F04385B004460D460026B1460427DFF854
:10286000A483A6884FF6C0700640684600F0F9FAC7
:10287000DDF80880E448B8FBF0F01FFA80F946EA7A
:102880000906A68020884FF6FE71084020800026A9
:10289000DE49286888420CD828684000B8FBF0F070
:1028A00087B2042F00DA04273E4309F10100208497
:1028B00027E0E8884BF6FF71884206D1286800EBD4
:1028C0004000B8FBF0F087B209E0286800EBC001D7
:1028D00001EB0010B8FBF0F087B247F48047C7F374
:1028E0000B0008B947F0010747F4004006434FF4D6
:1028F000967009FB00F04FF47A7190FBF1F0401CE8
:102900002084A683208840F00100208026884FF68E
:10291000F5300640A8886989084306432680A889BF
:1029200029890843208105B0BDE8F08341F2883150
:102930000160002181804BF6FF71C180002101817F
:1029400041814FF480418181704721B1028842F07A
:102950000102028004E002884FF6FE731A400280F2
:10296000704721B1828842F40062828004E082884C
:102970004FF2FF731A408280704721B1828842F47F
:102980008052828004E082884EF6FF731A40828073
:10299000704721B1028842F48072028004E002880C
:1029A0004FF6FF631A400280704721B1028842F45B
:1029B0000072028004E002884FF6FF531A40028042
:1029C000704721B1028842F48062028004E00288EC
:1029D0004FF6FF331A40028070470A460021818972
:1029E0004FF60173194002F0FE03194381817047CD
:1029F00021B1828942F00102828104E082894FF68E
:102A0000FE731A408281704721B1028842F0400271
:102A1000028004E002884FF6BF731A4002807047BC
:102A20001AB183880B43838002E083888B438380C1
:102A30007047018270470146088AC0B2704712B1E0
:102A400041F0010102E04FF6FE7319400182704728
:102A500008B50246002000900092009808440090BB
:102A60000098008808BD21B1028842F4004202802B
:102A700003E00288C2F30E0202807047B1F5006FD6
:102A800004D1028842F40062028004E002884FF21E
:102A9000FF731A4002807047B1F5005F04D10288CD
:102AA00042F40052028004E002884DF6FF731A409F
:102AB0000280704721B1028842F48052028004E013
:102AC00002884EF6FF731A4002807047B1F5006F1E
:102AD00004D1028842F40062028004E002884FF2CE
:102AE000FF731A400280704721B1028842F0200231
:102AF000028004E002884FF6DF731A4002807047BC
:102B00000146088B0012704721B1028842F0100282
:102B1000028004E002884FF6EF731A40028070478B
:102B200021B9028842F08002028004E002884FF658
:102B30007F731A4002807047B1F5804F05D0828BB9
:102B40004BF6FF731A40828303E0828B42F480428B
:102B50008283704770B502460024002500230020C0
:102B6000958A138B1B0445EA030626F07F4404EA8A
:102B700001068E4201D1012000E0002070BD10B599
:102B800001460020002300228B8A0A8B120443EAAC
:102B9000020424F07F4010BD0CB502460020002343
:102BA0000193009300920B0F019321F07F41019B51
:102BB0001BB1009B1433009303E0090C009B1833F6
:102BC0000093009B1B680B400BB1012000E000202C
:102BD0000CBD002221F07F42D3438382704730B581
:102BE000024600200023948801F0E06504EA1543C2
:102BF00021F07F41948A0C4054B14BB1012008E090
:102C00000054004000127A0040420F00A0860100EC
:102C1000002030BD002221F07F42D34383827047E1
:102C20000E49086070470D49486070470B4988603D
:102C300070474AF6AA200949086070474CF6CC4014
:102C400006490860704701460020044AD2680A40DD
:102C50000AB1012000E00020704700000030004071
:102C6000DF48006840F00100DD4908600846406820
:102C7000DC490840DA49486008460068DA490840FB
:102C8000D74908600846006820F48020086008469C
:102C9000406820F4FE0048604FF41F0088607047D1
:102CA000CF49096821F48031CD4A11601146096885
:102CB00021F480211160B0F5803F03D0B0F5802F62
:102CC0000ED106E0C649096841F48031C44A11605A
:102CD00007E0C349096841F4A021C14A116000E03E
:102CE00000BF00BF704710B501460022002300203E
:102CF0004A11012A02D1BA4C236806E0022A02D105
:102D0000B74C236A01E0B64C636A01F01F0201244C
:102D100094401C400CB1012000E0002010BD38B5EB
:102D2000002000900024002500BF3120FFF7DBFFCA
:102D300005460098401C00900098B0F5A06F01D0A7
:102D4000002DF2D03120FFF7CEFF08B1012400E0C2
:102D50000024204638BD01460020A14A106820F01A
:102D6000F80040EAC10010607047A0490860704751
:102D7000024600209A4B586820F47C1042EA010376
:102D80001843974B5860704798490866704701464A
:102D90000020934A506820F00300084350607047B9
:102DA0008F48406800F00C007047014600208C4AB4
:102DB000506820F0F0000843506070470146002042
:102DC000874A506820F4E06008435060704701462D
:102DD0000020834A506820F4605040EAC1005060EF
:102DE000704729B17E4A527A02437D4B5A7204E001
:102DF0007B4A527A82437A4B5A7270477B49D83168
:102E00000860704701460020754A506820F4404031
:102E10000843506070470021714A20321170704A97
:102E200082F82010012802D004280AD104E00121F0
:102E30006B4A2032117005E00521694A2032117079
:102E400000E000BF00BF70476949086070476449EF
:102E5000096A0143624A1162704765494439086052
:102E6000704730B500210022002400235C4D6D68BE
:102E700005F00C0121B1042905D0082923D105E072
:102E80005C4D056022E05B4D05601FE0544D6D68B0
:102E900005F47012524D6D6805F48034022505EB7F
:102EA00092421CB9544D554305600BE04C4D6D6882
:102EB00005F400351DB1504D5543056002E04D4D00
:102EC0005543056002E04B4D056000BF00BF444D17
:102ED0006D6805F0F0010909484D6B5C0568DD403F
:102EE00045603F4D6D6805F4E061090A434D6B5C38
:102EF0004568DD4085603A4D6D6805F46051C90A4A
:102F00003E4D6B5C4568DD40C560354D6D6805F430
:102F10004041890B3A4D6B5CC568B5FBF3F5056123
:102F200030BD29B12E4A526902432D4B5A6104E04B
:102F30002B4A526982432A4B5A61704729B1284A69
:102F400092690243264B9A6104E0254A92698243C2
:102F5000234B9A61704729B1214AD2690243204B21
:102F6000DA6104E01E4AD26982431D4BDA61704780
:102F700029B11B4AD2680243194BDA6004E0184AAF
:102F8000D2688243164BDA60704729B1144A12693D
:102F90000243134B1A6104E0114A12698243104B39
:102FA0001A61704712494039086070470F49C86478
:102FB00070470B49C87170470948406A40F08070FB
:102FC00007494862704701460020054A92680A4056
:102FD0000AB1012000E00020704701498872704763
:102FE000001002400000FFF8FFFFF6FE0000424222
:102FF0008004424200127A0000093D0029010020AD
:103000003901002010B50446FE48844208D1012150
:10301000C014FFF7ADFF0021E014FFF7A9FFC4E0E3
:10302000B4F1804F08D101210846FFF7AEFF00211F
:103030000120FFF7AAFFB8E0F348844208D101213C
:103040000220FFF7A2FF00210220FFF79EFFACE065
:10305000EE48844208D101210420FFF796FF0021A9
:103060000420FFF792FFA0E0E948844208D1012143
:103070000820FFF78AFF00210820FFF786FF94E071
:10308000E448844208D101211020FFF77EFF00218F
:103090001020FFF77AFF88E0DF48844208D1012141
:1030A0002020FFF772FF00212020FFF76EFF7CE059
:1030B000DA48844208D101214014FFF759FF00216A
:1030C0006014FFF755FF70E0D548844209D1012113
:1030D000C804FFF74DFF00214FF40020FFF748FF21
:1030E00063E0D048844209D101210805FFF740FF81
:1030F00000214FF48010FFF73BFF56E0CA4884429E
:1031000009D101214805FFF733FF00214FF40010DA
:10311000FFF72EFF49E0C548844208D10121402035
:10312000FFF733FF00214020FFF72FFF3DE0C048AD
:10313000844208D101218020FFF727FF0021802051
:10314000FFF723FF31E0BB48844208D101218015FD
:10315000FFF71BFF0021A015FFF717FF25E0B6487A
:10316000844209D101210804FFF702FF00214FF436
:103170008030FFF7FDFE18E0B048844209D10121FC
:103180004804FFF7F5FE00214FF40030FFF7F0FE92
:103190000BE0AB48844208D101218804FFF7E8FE28
:1031A00000214FF48020FFF7E3FE10BD00220288CB
:1031B000944B98420ED0994B98420BD0B0F1804F6F
:1031C00008D0914B984205D0904B984202D0904B3A
:1031D000984204D14FF68F731A404B881A438D4B97
:1031E000984207D08C4B984204D04FF6FF431A40C8
:1031F000CB881A4302808B8883850B880385814B9B
:1032000098420BD0854B984208D08B4B984205D002
:103210008A4B984202D08A4B984201D10B7A03869E
:1032200001238382704770B5002400220023058C9F
:103230004FF6FE7635400584028C8388048B4FF66A
:103240008F752C40B51E2C400D882C43751E2A40CE
:103250000D892A434D882A436A4DA8420BD06F4DF1
:10326000A84208D0744DA84205D0744DA84202D09F
:10327000734DA84213D14FF6F7752A404D892A4362
:103280004FF6FB752A408D882A434FF6FF652B4089
:103290004FF6FF552B408D892B43CD892B438380DF
:1032A0000483CD888586028470BD70B50024002219
:1032B0000023058C4FF6EF7635400584028C838819
:1032C000048B48F6FF752C404FF6FF452C400D88C7
:1032D0004FF6FF7606EA05252C434FF6DF752A40A8
:1032E0000D8906EA05152A434D8806EA05152A4385
:1032F000444DA84202D0494DA8421DD14FF67F75DA
:103300002A404D894FF6FF7606EA05152A434FF607
:10331000BF752A408D8806EA05152A434FF6FF350A
:103320002B404FF2FF752B408D8906EA85052B4314
:10333000CD8906EA85052B4383800483CD880587E4
:10334000028470BD70B5002400220023058C4FF666
:10335000FF6635400584028C8388848B4FF68F7519
:103360002C404FF6FC752C400D882C434FF6FF5532
:103370002A400D894FF6FF7606EA05252A434D8837
:1033800006EA05252A431F4DA84202D0234DA84234
:103390001DD14FF2FF752A404D894FF6FF7606EAA0
:1033A00005252A434FF6FF352A408D8806EA052574
:1033B0002A434EF6FF752B404DF6FF752B408D8945
:1033C00006EA05152B43CD8906EA05152B438380B4
:1033D0008483CD888587028470BD70B50022002368
:1033E0000024058C4EF6FF7635400584038C8488D6
:1033F000828B48F6FF752A404FF6FF452A400D881C
:1034000020E00000002C01400004004000080040C3
:10341000000C004000100040001400400034014047
:10342000004C014000500140005401400018004091
:10343000001C0040002000400040014000440140CA
:10344000004801404FF6FF7606EA05252A434DF66F
:10345000FF752B400D8906EA05352B434D8806EA9A
:1034600005352B43FA4DA84202D0FA4DA84208D1A7
:103470004BF6FF752C408D894FF6FF7606EA8515D1
:103480002C4384808283CD88A0F84050038470BD93
:10349000828B4FF2FF331A408283828B4FF6FF7389
:1034A00003EA01231A4382837047F0B50C461546A0
:1034B000002200210026078C4EF6FF7C07EA0C074D
:1034C0000784828B018C4FF6FF7707EA043640F6BB
:1034D000FF473A404FF6FF7707EA05273A434FF692
:1034E000FF7707EA03373A43D94FB8420ED0D94F96
:1034F000B8420BD0B0F1804F08D0D74FB84205D0BA
:10350000D64FB84202D0D64FB84206D14DF6FF771B
:10351000394046F48057394305E047F6FF573940B4
:1035200044F48057394382830184F0BD828B4FF687
:10353000F3731A408283828B0A4382837047F0B50B
:103540000C461546002200210026078C4FF6FF6C22
:1035500007EA0C070784828B018C4FF6FF7707EA96
:1035600004264FF60C773A404FF6FF7707EA031729
:103570002F433A43B64FB8420ED0B64FB8420BD0A5
:10358000B0F1804F08D0B44FB84205D0B34FB84225
:1035900002D0B34FB84206D14FF6FF57394046F438
:1035A0008077394305E04FF2FF57394044F4807784
:1035B000394382830184F0BD028B4FF2FF331A40FE
:1035C0000283028B4FF6FF7303EA01231A4302833F
:1035D0007047F0B50C461546002200210026078CE6
:1035E0004FF6EF7C07EA0C070784028B018C4FF63D
:1035F000FF7707EA041640F6FF473A404FF6FF7799
:1036000007EA03373A434FF6FF7707EA05273A43BD
:103610008F4FB8420ED08F4FB8420BD0B0F1804FD1
:1036200008D08D4FB84205D08C4FB84202D08C4F95
:10363000B84206D14FF6DF77394046F010073943DC
:1036400005E04FF65F77394044F0100739430283B5
:103650000184F0BD028B4FF6F3731A400283028B94
:103660000A4302837047F0B50C461546002200213C
:10367000068C4FF6FE773E400684028B018C4FF697
:103680000C7632407E1C06EA03162E433243704EFF
:10369000B0420ED06F4EB0420BD0B0F1804F08D088
:1036A0006D4EB04205D06D4EB04202D06C4EB0426D
:1036B00006D14FF6FD76314044F00106314305E076
:1036C0004FF6F576314044F0010631430283018420
:1036D000F0BD70B505460C465D4885420ED05D488C
:1036E00085420BD0B5F1804F08D05B48854205D0AC
:1036F0005A48854202D05A48854200D100E000BFB6
:10370000208850B92389A28861882846FFF7ABFF3B
:10371000E1882846FFF79EFF25E0208804280AD18B
:103720002389A28861882846FFF753FFE18828464D
:10373000FFF742FF17E0208808280AD12389A288D2
:1037400061882846FFF7FBFEE1882846FFF7EEFE7A
:1037500009E02389A28861882846FFF7A6FEE18850
:103760002846FFF795FE70BD2DE9F04105460C4651
:1037700000260127608808B9022600E00026A088FC
:10378000012801D1022700E001272088A0B9238960
:10379000A28861882846FFF766FFE1882846FFF780
:1037A00059FF23893A4631462846FFF712FFE18840
:1037B0002846FFF701FF13E02389A2886188284685
:1037C000FFF707FFE1882846FFF7F6FE23893A4610
:1037D00031462846FFF747FFE1882846FFF73AFFC2
:1037E000BDE8F0810A884B881A438B881A43CB883E
:1037F0001A430B891A434B891A438B891A43A0F841
:10380000442070474FF6FF71818000210180C18004
:103810004180017270470021018041808180C18018
:10382000018141818181C1817047002101804180F6
:10383000012181800021C180018170470021018028
:1038400041808180C1800181418181817047000078
:10385000002C0140003401400004004000080040FA
:10386000000C004021B1028842F00102028004E015
:1038700002884FF6FE731A400280704731B1B0F8EB
:10388000442042F40042A0F8442005E0B0F844206F
:10389000C2F30E02A0F8442070471AB183890B438B
:1038A000838102E083898B438381704781827047E3
:1038B00041EA0203A0F8483070471AB183890B43EC
:1038C000838102E083898B438381704701894FF6AE
:1038D000F8721140018170470A46002101894FF6B4
:1038E0008F73194011430181704730B504460D466E
:1038F00029462046FFF7F0FF208940F0070020818D
:1039000030BD2DE9F04104460D4616461F46602D98
:1039100006D13B46012231462046FFF75AFE05E01C
:103920003B46012231462046FFF79DFE29462046B0
:10393000FFF7D2FF208940F007002081BDE8F08129
:1039400030B50C4600210189C9B24FF6FF7505EA72
:103950000325154325432943018130BD2DE9F0415D
:1039600005460E4617469846002443463A463146D9
:103970002846FFF7E5FF2C894FF6F870044044F025
:1039800007044FF68F70044044F070042C81BDE8AA
:10399000F081F0B504460D4616461F463B463246BA
:1039A00029462046FFF7CCFF208940F48040208143
:1039B000F0BD0185828270470A46002101884FF6DA
:1039C0008F731940114301807047F0B50C461546BE
:1039D0001E460021002200230189028B038C4FF632
:1039E000F877394021434FF6FC473A4040F201173F
:1039F0003A434FF6DD773B404FF6FF7707EA06176D
:103A00002F433B43018102830384F0BD0A4600211A
:103A1000018B4FF68F7319401143018370470A469B
:103A20000021018B48F6FF7319404FF6FF7303EA3C
:103A300002231943018370470A460021818B4FF608
:103A40008F7319401143818370470A460021818B8F
:103A500048F6FF7319404FF6FF7303EA0223194338
:103A60008183704721B1028842F08002028004E025
:103A700002884FF67F731A400280704721B1828816
:103A800042F00402828004E082884FF6FB731A4001
:103A90008280704721B1828842F00802828004E06F
:103AA00082884FF6F7731A408280704721B182886E
:103AB00042F00102828004E082884FF6FE731A40D1
:103AC000828070470A460021018B4FF6F773194038
:103AD0001143018370470A460021018B4FF2FF73A7
:103AE00019404FF6FF7303EA02231943018370471D
:103AF0000A460021818B4FF6F773194011438183E9
:103B000070470A460021818B4FF2FF7319404FF630
:103B1000FF7303EA02231943818370470A46002199
:103B2000018B4FF6FB7319401143018370470A461E
:103B30000021018B4FF6FF3319404FF6FF7303EA64
:103B400002231943018370470A460021818B4FF6F7
:103B5000FB7319401143818370470A460021818B12
:103B60004FF6FF3319404FF6FF7303EA0223194360
:103B7000818370470A460021018B4FF67F731940FD
:103B80001143018370470A460021018BC1F30E01E6
:103B90004FF6FF7303EA02231943018370470A4675
:103BA0000021818B4FF67F73194011438183704749
:103BB0000A460021818BC1F30E014FF6FF7303EA21
:103BC00002231943818370470A460021018C4FF676
:103BD000FD7319401143018470470A460021018C8E
:103BE0004FF6F77319401143018470470A460021CC
:103BF000018C4FF6DF7319404FF6FF7303EA02138F
:103C00001943018470470A460021018C4FF67F73E7
:103C100019404FF6FF7303EA0213194301847047FA
:103C20000A460021018C4FF6FF5319404FF6FF73EF
:103C300003EA02231943018470470A460021018CDC
:103C40004FF2FF7319404FF6FF7303EA0223194343
:103C5000018470470A460021018C4DF6FF7319401C
:103C60004FF6FF7303EA023319430184704730B5FE
:103C7000002301248C40A3B2048C9C430484048C54
:103C800002FA01F5ADB22C43048430BD30B50023F7
:103C900004248C40A3B2048C9C430484048C02FA58
:103CA00001F5ADB22C43048430BD70B5034600204D
:103CB00000241846183001258D40ACB21D8CA54358
:103CC0001D8409B1082909D100EB6100056825F0C0
:103CD000700505600568154305600EE00D1FC5F30E
:103CE0004E052844056825F4E045056005684FF653
:103CF000FF7606EA02263543056070BD21B10288D1
:103D000042F00202028004E002884FF6FD731A407E
:103D10000280704721B1028842F00402028004E070
:103D200002884FF6FB731A400280704721B18288E7
:103D300042F08002828004E082884FF67F731A404E
:103D40008280704702884FF6F7731A40028002881B
:103D50000A430280704782884FF68F731A40828030
:103D600082880A438280704702894FF6F8731A40AE
:103D7000028102890A430281704702894FF67F73EC
:103D80001A40028102890A43028170478184704788
:103D900081857047818670470187704781877047AA
:103DA000A0F84010704702884FF6FF431A40028087
:103DB00002880A43028070470146888E7047014698
:103DC000088F70470146888F70470146B1F8400060
:103DD00070470146888C70470146088D704702463F
:103DE0000020138A0B400BB1012000E00020704737
:103DF000CA430282704730B50246002000230024E7
:103E0000158A05EA0103958905EA010413B10CB18D
:103E1000012000E0002030BDCA430282704700004C
:103E200010B50446FB48844209D101218803FFF7FD
:103E30009FF800214FF48040FFF79AF832E0F648EF
:103E4000844209D101214804FFF79FF800214FF473
:103E50000030FFF79AF825E0F048844209D10121AB
:103E60008804FFF792F800214FF48020FFF78DF8C7
